:0200000480007A
:100000006F008004732F2034930F80006308FF0378
:10001000930F90006304FF03930FB0006300FF038E
:10002000130F000063040F0067000F00732F2034CC
:1000300063540F006F00400093E19153171F0000BD
:1000400023223FFC6FF09FFF93000000130100008C
:10005000930100001302000093020000130300004C
:100060009303000013040000930400001305000034
:10007000930500001306000093060000130700001C
:100080009307000013080000930800001309000004
:1000900093090000130A0000930A0000130B0000EC
:1000A000930B0000130C0000930C0000130D0000D4
:1000B000930D0000130E0000930E0000130F0000BC
:1000C000930F0000732540F16310050097020000B4
:1000D000938202017390523073500018970200000F
:1000E00093824202739052309B021000939252030B
:1000F0009382F2FF7390023B9302F0017390023AF5
:100100007350403097020000938242017390523046
:10011000735020307350303093010000970200007C
:10012000938282EE73905230130510001315F5017F
:10013000635C05000F00F00F930110009308D005D9
:10014000130500007300000093020000638A0200A0
:1001500073905210B7B200009B82921073902230BD
:100160007350003097020000938242017390123462
:10017000732540F1730020309301200093000000AC
:100180001301100063C620006318302A6316300084
:10019000E3CE20FE6312302A930130009300F0FF7B
:1001A0001301100063C62000631830286316300066
:1001B000E3CE20FE63123028930140009300E0FF5D
:1001C0001301F0FF63C62000631830266316300069
:1001D000E3CE20FE631230269301500093001000FE
:1001E0001301000063C42000631430006316302440
:1001F000E3CE20FE93016000930010001301F0FF96
:1002000063C420006314300063183022E3CE20FE64
:10021000930170009300F0FF1301E0FF63C420001E
:1002200063143000631A3020E3CE20FE9301800077
:10023000930010001301E0FF63C42000631430003A
:10024000631C301EE3CE20FE9301900013020000D9
:10025000930000001301F0FF63C0201E1302120080
:1002600093022000E31652FE9301A0001302000047
:10027000930000001301F0FF1300000063CE201A6A
:100280001302120093022000E31452FE9301B00007
:1002900013020000930000001301F0FF13000000A0
:1002A0001300000063CA20181302120093022000FA
:1002B000E31252FE9301C0001302000093000000FD
:1002C000130000001301F0FF63C820161302120090
:1002D00093022000E31452FE9301D00013020000A9
:1002E00093000000130000001301F0FF1300000052
:1002F00063C420141302120093022000E31252FE82
:100300009301E000130200009300000013000000BE
:10031000130000001301F0FF63C02012130212004B
:1003200093022000E31252FE9301F000130200003A
:10033000930000001301F0FF63C0201013021200AD
:1003400093022000E31652FE930100011302000005
:10035000930000001301F0FF1300000063CE200C97
:100360001302120093022000E31452FE93011001C5
:1003700013020000930000001301F0FF13000000BF
:100380001300000063CA200A130212009302200027
:10039000E31252FE930120011302000093000000BB
:1003A000130000001301F0FF63C8200813021200BD
:1003B00093022000E31452FE930130011302000067
:1003C00093000000130000001301F0FF1300000071
:1003D00063C420061302120093022000E31252FEAF
:1003E000930140011302000093000000130000007D
:1003F000130000001301F0FF63C020041302120079
:1004000093022000E31252FE93001000634A100092
:100410009380100093801000938010009380100050
:1004200093801000938010009303300093015001DB
:1004300063947000631030020F00F00F63800100BE
:100440009391110093E111009308D00513850100E9
:10045000730000000F00F00F930110009308D00507
:100460001305000073000000731000C000000000BE
:0C04700000000000000000000000000080
:1010000000000000000000000000000000000000E0
:1010100000000000000000000000000000000000D0
:1010200000000000000000000000000000000000C0
:1010300000000000000000000000000000000000B0
:081040000000000000000000A8
:040000058000000077
:00000001FF
